:10000000020003758143120146E582600302006F1E
:10001000780079007A007B007C007D00EC4D601C4C
:1000200088828983E493A3A882A9838A828B83F040
:10003000A3AA82AB831CBCFFE31D80E07582007520
:1000400083007C007D00EC4D600AE4F0A31CBCFF43
:10005000F51D80F27582007583007C007D00EC4DFB
:10006000600AE4F0A31CBCFFF51D80F2120115121A
:1000700002CE80FE1B5B324A00414443207465730C
:10008000742070726F6772616D0A46696C653A2000
:1000900025730A436F6D70696C65643A2025732C73
:1000A0002025730A0A00433A5C55736572735C65D8
:1000B0007468616E5C4F6E654472697665202D20B0
:1000C0005542435C4465736B746F705C4C61623580
:1000D0005C7A65726F2063726F73732064657465F8
:1000E0006374696F6E2E63004D617220203620327A
:1000F0003032340032313A30353A343900564050DB
:10010000322E323A25660D000A00564050322E310A
:100110003A25660D00750A00750B00750C00750D0B
:1001200000750E00750F0075100075110075120036
:100130007513007514007515007516007517007598
:1001400018007519002275A7007597DE7597AD75B3
:10015000FF8075EF0675A71075C12075A70075A9FA
:100160000075A900E5A930E7FB75A90375A903E5AA
:10017000A930E7FB43A41075E10175E20075E34087
:10018000759810758DE6858D8B53890F438920D224
:100190008ED2997582002275A700C2EF75B2807564
:1001A000BC2075B91E75E80075DF3F75B300D2EF4E
:1001B00022AA82438E407592B87593FF85929485EA
:1001C00093957591047B00C3EB9A500BE59130E752
:1001D000FB53917F0B80F075910022AA82AB837C48
:1001E000007D00C3EC9AED9B502B7E00BE040050B6
:1001F0001D7582FAC002C003C004C005C00612010A
:10020000B1D006D005D004D003D0020E80DE0CBCE5
:1002100000D10D80CE22AA82851BF005F0740180EA
:100220000225E0D5F0FBFB75A720BA0002800ABAD0
:100230000102800FBA021E8014EBF4FA52F1EB4275
:10024000D48012EBF4FA52F2EB42D58008EBF4FAC8
:1002500052F3EB42CC75A700228582BBC2EDD2ECF3
:1002600030EDFD85BD8285BE832212025912044BFA
:10027000AA82AB83ACF0FDC002C003C004C00590ED
:10028000923A75F0537440120487AA82AB83ACF0A3
:10029000FDE58124FCF581E4C0E074FCC0E0747FDE
:1002A000C0E07446C0E08A828B838CF0ED1205605A
:1002B000AA82AB83ACF0FDE58124FCF5818A828BB8
:1002C000838CF0ED225389F0438901C28C22120203
:1002D000C59001F41201DB7474C0E07400C0E074D6
:1002E00080C0E012053F15811581158174F4C0E0CE
:1002F0007400C0E07480C0E074E8C0E07400C0E046
:100300007480C0E074A6C0E07400C0E07480C0E0F7
:100310007479C0E07400C0E07480C0E012053FE56D
:100320008124F4F581751B01758202120216751B7A
:100330000275820212021612019775820F12026A6A
:10034000AA82AB83ACF0FDE4C0E0C0E0C0E0C0E056
:100350008A828B838CF0ED120457AA82E58124FCFB
:10036000F581EA602C75820F12026AAA82AB83AC17
:10037000F0FDC002C003C004C00574FDC0E07400FD
:10038000C0E07480C0E012053FE58124F9F581806A
:10039000A9D2B27408C0E07401C0E07480C0E01259
:1003A000053F15811581158175820E12026AAA8298
:1003B000AB83ACF0FDE4C0E0C0E0C0E0C0E08A8206
:1003C0008B838CF0ED120457AA82E58124FCF58121
:1003D000EA602C75820E12026AAA82AB83ACF0FD31
:1003E000C002C003C004C005740AC0E07401C0E0CC
:1003F0007480C0E012053FE58124F9F58180A9C22F
:10040000B27408C0E07401C0E07480C0E012053F1F
:1004100015811581158175820F12026AAA82AB833C
:10042000ACF0FDEA4B4C8DF0C2F745F060E8758208
:100430000E12026AAA82AB83ACF0FDEA4B4C8DF03F
:10044000C2F745F0600302033A80E3E4AC83AB8279
:10045000FAF9748E020688FFA88118181206B0D225
:10046000D133E6400730E70B7582012220E706759D
:10047000820022C2D1120692E97003F5822230D1A5
:1004800001B3E433F5822212075DBC00030206FCCF
:10049000EF60FA30D502B2D1E583B4FF0302071250
:1004A000E582B4FF03020712258340072482400B34
:1004B0000206FC2483145003020712F582EA8DF031
:1004C000A4A8F0EA8EF0A428F8E435F0F9EB8DF05A
:1004D000A428E935F0F9E433CA8FF0A429F9EA3504
:1004E000F0FAEBF88EF0A429F9EA35F0FAE433FBE0
:1004F000EC8DF0A429F9EA35F0FAE43BFBE88FF043
:10050000A42AFAEB35F0FBE433CCFD8EF0A42AFAF2
:10051000EB35F0FBE43CFCED8FF0A42BFBEC35F06D
:10052000FC20E70312072A0206DB0211178582303E
:1005300085833185F032851A3390052A020B6AC013
:1005400008858108E50824FBF533E50824FBF886D7
:100550003008863108863290052A120B6AD00822AC
:1005600012075D30D502B2D1BF0009BC00030207FB
:100570001F020712BC00030206FCE583B4FF0BE573
:1005800082B4FF0302071F0206FCE582B4FF0302E8
:100590000712C395835007247F400B0206FC24807A
:1005A000145003020712C0E0E4CCCBCAF98D1B8EB5
:1005B0001C8F1DEF54F0C4F51E758306851EF0EBED
:1005C00084F582E9C4F9EAC4FAEBC4FBEC540FC425
:1005D0007803D6FC18EBD6FB18EAD6FA8582F0ED44
:1005E000A4A8F0FD8582F0EEA428FEE435F0F8859D
:1005F00082F0EFA428FFE435F0F8E99DF9EA9EFACD
:10060000EB9FFBEC98FCAD1BAE1CAF1D30E710154B
:1006100082E92DF9EA3EFAEB3FFBE43CFC80EDC0B9
:1006200082D58398C3E933F9EA33FAEB33FBEC3331
:10063000FCC3E99DEA9EEB9FEC9400B3E413F9D070
:1006400002D0E0C44AFAD003D0E0C44BFBD004D0BF
:10065000E0F5F0540FC44CFCD082158230F40FD377
:10066000EC13FCEB13FBEA13FAE913F90582E9300A
:10067000E70A74012AFAE43BFBE43CFC0206F3FCC3
:10068000ABF0AA83A982749EC2D1F58212072A0216
:1006900006DB7901AA82E68F82B5821318E6B5F0EF
:1006A0000E18E6B5830918E68A82B582027900221F
:1006B000B4800FE5F0700AE5837006E58270027F72
:1006C00000EFB6801518B6001018B6000B18B6006B
:1006D0000608080876002208080822B98003EA13F1
:1006E000B34010EA2401FAE43BFBE43CFC50047CF8
:1006F000800582BC000EBB000BBA0008E4F5F0F5E3
:1007000083F58222A2D1E582138CF092F78B838A43
:100710008222E4F583F58275F080F4A2D11322E4FD
:10072000F583F58275F0C0747F227804EC7011E5D2
:100730008224F8500AF582E4C9CACBFCD8EF22EC37
:100740007820058220E713D5820122C3E933F9EA34
:1007500033FAEB33FBEC33FCD8EA158222AA82ABE6
:1007600083A2F73392D16002D2F7F582ACF0E58133
:1007700024F9F8E6FD08E6FE0886F008E6A2F7335D
:1007800092D56002D2F7F583AFF022AA82749CC0A2
:10079000E07407C0E0C022C0238A82220529E4B5A4
:1007A0002902052A22AA8274302AFA24C6500A7421
:1007B000072AFA3000034302208A8202078BE5826F
:1007C000FAC4540FF582C0021207A5D002740F5A62
:1007D000F5820207A5AA24AB25AC26AD27AE287565
:1007E0002F20EE2EFEED235401FF4206EA2AFAEBFB
:1007F00033FBEC33FCED33FDC3EE952B4008EEC329
:10080000952BFE430201D52FD98A248B258C268D6A
:10081000278E28227840E624D075F00AA4FA784181
:10082000E624D02AFA783F8603BB2D04C3E49AFA63
:10083000752B01C3E464808AF063F08095F0502941
:10084000752F038A0374F6252F401C052BE52F1402
:100850002434F8E52F2434F98704A604772E1BEB03
:10086000FA6004052F80DE8B02EA30E70D783586CA
:10087000037836A6037835762E0AE52D600AE52D35
:1008800004FB252BF52B8005300B02052B783486D5
:1008900003E4BB2D0104FB700620060330070205AC
:1008A0002B30040302095B300557EB600C75822D79
:1008B000C00212078BD002801C30060C75822BC040
:1008C0000212078BD002800D30070A758220C00209
:1008D00012078BD00278358604BC2E0C758230C08E
:1008E0000212078BD002152CAC2C152CC3E52B9CC7
:1008F000400302099F758230C00212078BD002802C
:10090000E7AC2C152CC3E52B9C500C758220C00243
:1009100012078BD00280EA78348604BC2D0C7582D5
:100920002DC00212078BD002801C30060C75822B62
:10093000C00212078BD002800D30070A758220C0DA
:100940000212078BD00278358604BC2E5275823095
:10095000C00212078BD002152C8044EB600E75820A
:100960002DC00212078BD002152C802030060E7588
:10097000822BC00212078BD002152C800F30070C7F
:10098000758220C00212078BD002152C78358603A1
:10099000BB2E0C758230C00212078BD002152C754D
:1009A0002F01C20DE52F2434F88603BB4503020A4C
:1009B0005CBB2E348A03C3E464808BF063F08095C3
:1009C000F0500F758230C00312078BD0031B8B02CF
:1009D00080E48B02D20DE52D7038200B03020A5CF7
:1009E00075822E12078B8074300D278A03EB30E757
:1009F0001FC3E46480852DF063F08095F0500C7582
:100A00008230C00312078BD003152D0B8B0280DDC3
:100A10008B02300D0EC3E46480852DF063F0809569
:100A2000F05021E52F2434F886038B82C002120790
:100A30008BD002300D0EE52F2434F88603BB2E0236
:100A40008002152D152CC3E46480852DF063F080A1
:100A500095F04003200D05052F0209A4C3E464802E
:100A6000852DF063F08095F0500A75823012078B67
:100A7000152D80E830040FAA2C152CEA6008758229
:100A80002012078B80F122E52D7003300B0D7407C7
:100A9000252DFAE52CC39AF52C8006E52C24FAF5D1
:100AA0002C752F0078348602BA2B0F20060C783470
:100AB0007620200705752F01052C200419AA2CC3C8
:100AC000E464808AF063F08095F0500A7582201209
:100AD000078B152C80E7C20DE52F2434F88602BA67
:100AE00000028069BA451F3000027665C3E4648065
:100AF000852DF063F08095F0500A75823012078BD7
:100B0000152D80E8D20DC3E52F9402E433FA70145A
:100B1000EA700EC3E46480852DF063F08095F040A8
:100B200003300D16E52F2434F886028A8212078BD3
:100B3000E52F24FD5012152D800E7402B52F0930BB
:100B40000B0675822E12078B052F020AD830041966
:100B5000AA2CC3E464808AF063F08095F0500A7593
:100B6000822012078B152C80E72285822285832321
:100B7000E4F529F52AAA30AB31AC328A828B838C1A
:100B8000F012112CFD74012AF530E43BF5318C3262
:100B9000EDFA7003021110BA25028003021108C297
:100BA00004C205C206C207C208C209C20AC20BC2F9
:100BB00001C202C203752B00752C00752DFFAB30EE
:100BC000AC31AD328B828C838DF012112CFAA3AB39
:100BD00082AC838B308C318D32BA25078A82120722
:100BE0008B80928A06BE3000402E8A06EE24C640D4
:100BF0002774FFB52D13E52C75F00AA4FEEA24D066
:100C00002EF52C70BFD20580BBE52D75F00AA4FE31
:100C1000EA24D02EF52D80ACBA2E0A74FFB52DA48F
:100C2000752D00809F8A06BE6100400E8A06EE2464
:100C30008540075302DFD2008002C200BA20028042
:100C400075BA2303020CC5BA2A03020CCABA2B02D6
:100C5000805FBA2D028055BA4202805FBA43030218
:100C60000D0FBA4403020E4ABA4503020E64BA4697
:100C700003020E60BA4703020E68BA4903020E4A25
:100C8000BA4C02803BBA4E03020E6CBA4F03020EFE
:100C900051BA5003020DE3BA5303020D33BA5503A0
:100CA000020E56BA5803020E5B020E96D204020BD5
:100CB000C4D206020BC4D207020BC4D209020BC471
:100CC000D20A020BC4D20B020BC474FFB52D203024
:100CD000090BE53314F88833862C020BC4E5332462
:100CE000FEF888338606088607188E2C020BC4305F
:100CF000090BE53314F88833862D020BC4E5332441
:100D0000FEF888338606088607188E2D020BC4303D
:100D1000090AE53314F888338602800FE53324FE90
:100D2000F888338603088604188B028A8212078BA0
:100D3000020E9BE53324FDF88833860308860408F9
:100D4000860518188B248C258D268B828C838DF03C
:100D5000121280AB82AC838B2E74FFB52D03852ECF
:100D60002D20041DC3E52E952C5016E52CC3952E81
:100D7000F52CAB2C152CEB600875822012078B80AC
:100D8000F18524828525838526F012112CFBFA60DB
:100D900029AB2D152DC3E464808BF063F08095F0B2
:100DA00050188A8212078BAB24AC25AD260BBB00F2
:100DB000010C8B248C258D2680C7200403020E9BFA
:100DC000C3E52E952C4003020E9BE52CC3952EF512
:100DD0002CAB2C152CEB7003020E9B758220120796
:100DE0008B80EEE53324FDF88833860308860408FB
:100DF000860518188B248C258D26E526FB30E70404
:100E00007A438013EB546060047A50800AEB30E63A
:100E1000047A4980027A588A82C00212078B75824E
:100E20003A12078B75823012078B75827812078B06
:100E3000D002BA4902800BBA500280068525821280
:100E400007BE8524821207BE8051D208752B0A8006
:100E50004A752B088045752B0A8040752B10803B06
:100E6000D2018037D2028033D203802FE53324FDB4
:100E7000F88833860308860408860518188B248CA6
:100E8000258D268B828C838DF0E529121267A3E5D0
:100E90002A12126780058A8212078B20010620021F
:100EA00003300370E53324FCF88833860308860496
:100EB0000886050886061818188B248C258D268E22
:100EC00027E524E525E526E5278B828C838DF0EE4A
:100ED00012114874FFB52D03752D06300327747F5A
:100EE0005527FB8B28E528EB2BFB8B28E52630E7E5
:100EF0000674014528F528E52824684006749925DC
:100F0000284002D202300206120A87020B7512082C
:100F100014020B75E52B7003020B757B3930092B1E
:100F2000E53314F88833E6FC3395E0FDFEFF8C24AE
:100F30008D258E268F2720085EAC247D007E007FC5
:100F4000008C248D258E268F27804C300A1FE53398
:100F500024FCF88833860408860508860608860778
:100F60001818188C248D258E268F27802AE5332487
:100F7000FEF88833860408860518ED3395E0FEFFF9
:100F80008C248D258E268F2720080CAC24AD257E41
:100F9000007F008E268F27300B43E524452545260C
:100FA000452760397408B52B0C758230C0031207D1
:100FB0008BD00380287410B52B23758230C00312A8
:100FC000078BD00330000C758278C00312078BD0DA
:100FD00003800A758258C00312078BD0033008259E
:100FE000AC24AD25AE26E527FF30E717C3E49CFC13
:100FF000E49DFDE49EFEE49FFF8C248D258E268FCC
:10100000278002C208752E00D20C8B00752800C004
:10101000001207D5D000200C0DE528C4FCE6FD4CDD
:10102000F61888038002A628052EB20CE524452573
:101030004526452770D68803E52C7003752C0120C2
:10104000051A200417E52E04FCC3952C500E75825A
:1010500020C00312078BD003152C80E930080E75D1
:10106000822DC00312078BD003152C8024E52E603F
:101070002030060E75822BC00312078BD003152C6F
:10108000800F30070C758220C00312078BD0031528
:101090002C20041EAC2C152CC3E52E9C50273005AB
:1010A000047C3080027C208C82C00312078BD0032A
:1010B00080E2C3E52E952C5009E52CC3952EF52C26
:1010C0008003752C008B00AB2E152EEB6022B20C2A
:1010D000200C0A08E6C4540FFB8B28800786037493
:1010E0000F5BF528852882C0001207A5D00080D7A5
:1010F000200403020B75AB2C152CEB7003020B754F
:1011000075822012078B80EE8A8212078B020B7584
:10111000852982852A8322AA82BA0A081099028028
:10112000FB75990D10990280FB8A992220F71430E3
:10113000F6148883A88220F507E6A8837583002229
:10114000E280F7E49322E022C0E0F845824583453F
:10115000F07009F5F0FBFCFDFE021216E823A2F781
:1011600092E0F8A982AA83D2F7ABF07C007E07C395
:10117000749798404074FF2EFE740A89F0A4F98594
:10118000F082740A8AF0A4FA85F083740A8BF0A4C2
:10119000FB740529F9EA3582FAEB3583FB740035D7
:1011A000F0FCC3EC13FCEB13FBEA13FAE913F908A8
:1011B000EC70EF80BAE8C3947FF88B838EF0E4FB89
:1011C000FCFDFEFF08C3E933F9EA33FAE58333F5A2
:1011D00083EB3BD4FBEC3CD4FCED3DD4FDEE3ED4A4
:1011E000FEEF3FD4FF602D05F074052BD4FBE43CEB
:1011F000D4FCE43DD4FDE43ED4FEE43FD4FF75824C
:1012000004C3EF13FFEE13FEED13FDEC13FCEB1321
:10121000FBD582EDD8AF7834D0E020E704762B8080
:1012200002762D087906E7C4540F4430F608B90653
:1012300003762E08E7540F4430F60819B902E77612
:101240004508E5F020E704762B8004762DF40408A9
:1012500075F00A844430F608E5F04430F608E4F608
:1012600090003475F0402220F71030F6118883A8E2
:101270008220F507F6A88375830022F280F7F0221A
:10128000AA82AB83ACF07D007E008A828B838CF0D7
:1012900012112CFFA3AA82AB83EF60070DBD00EAF9
:1012A0000E80E78D828E8322000000000000000087
:00000001FF
